:020000040800F2
:10000000C0040020050100080D0100080F010008D0
:10001000110100081301000815010008000000008C
:1000200000000000000000000000000017010008B0
:1000300019010008000000001B010008D904000895
:100040001F0100081F0100081F0100081F01000810
:100050001F0100081F0100081F0100081F01000800
:100060001F0100081F0100081F0100081F010008F0
:100070001F0100081F0100081F0100081F010008E0
:100080001F0100081F0100081F0100081F010008D0
:100090001F0100081F0100081F0100081F010008C0
:1000A0001F0100081F0100081F0100081F010008B0
:1000B00085050008890500081F0100081F010008C8
:1000C0001F0100081F0100081F0100081F01000890
:1000D0001F010008F50700081F0100081F010008A4
:1000E0001F0100081F0100081F010008DFF810D0E1
:1000F00000F02CF8004800472D120008AFF30080F4
:10010000C00400200648804706480047FEE7FEE797
:10011000FEE7FEE7FEE7FEE7FEE7FEE7FEE7FEE7B7
:1001200025050008ED00000840EA01039B0703D005
:1001300009E008C9121F08C0042AFAD203E011F826
:10014000013B00F8013B521EF9D27047064C074DA7
:1001500006E0E06840F0010394E807009847103497
:10016000AC42F6D3FFF7C6FF7813000898130008D7
:100170002DE9F0410246002500260020002300243E
:10018000002791F803C00CF00F0591F803C00CF0A4
:10019000100CBCF1000F03D091F802C04CEA050529
:1001A00091F800C0BCF1000F31D0146800202BE0A2
:1001B0004FF0010C0CFA00F3B1F800C00CEA030692
:1001C0009E4220D183004FF00F0C0CFA03F7BC4382
:1001D00005FA03FC4CEA040491F803C0BCF1280FB3
:1001E00006D14FF0010C0CFA00FCC2F814C00AE072
:1001F00091F803C0BCF1480F05D14FF0010C0CFA87
:1002000000FCC2F810C0401C0828D1D31460B1F81B
:1002100000C0BCF1FF0F34DD546800202EE000F177
:10022000080C4FF0010808FA0CF3B1F800C00CEA12
:1002300003069E4221D183004FF00F0C0CFA03F706
:10024000BC4305FA03FC4CEA040491F803C0BCF17A
:10025000280F05D100F1080C08FA0CF8C2F8148038
:1002600091F803C0BCF1480F07D100F1080C4FF022
:10027000010808FA0CF8C2F81080401C0828CED3F8
:100280005460BDE8F081000002490143024A116058
:10029000704700000000FA050CED00E029B1064AA5
:1002A000D2690243044BDA6104E0034AD269824313
:1002B000014BDA61704700000010024029B1064A84
:1002C00012690243044B1A6104E0034A1269824333
:1002D000014B1A61704700000010024029B1064A24
:1002E00092690243044B9A6104E0034A9269824393
:1002F000014B9A61704700000010024029B1064A84
:10030000D2680243044BDA6004E0034AD2688243B5
:10031000014BDA60704700000010024030B5002148
:100320000022002400232D4D6D6805F00C0121B141
:10033000042905D0082923D105E0294D056022E0D4
:10034000274D05601FE0254D6D6805F47012234DA3
:100350006D6805F48034022505EB92421CB9214DED
:10036000554305600BE01D4D6D6805F400351DB16A
:100370001C4D5543056002E0194D5543056002E0F0
:10038000174D056000BF00BF144D6D6805F0F0010A
:100390000909154D6B5C0568DD4045600F4D6D68C2
:1003A00005F4E061090A104D6B5C4568DD4085602D
:1003B0000A4D6D6805F46051C90A0B4D6B5C4568C8
:1003C000DD40C560054D6D6805F44041890B074D62
:1003D0006B5CC568B5FBF3F5056130BD00100240EC
:1003E00000127A0000093D003C0000204C00002073
:1003F00010B500F001F810BD0CB500200190009080
:100400003348006840F480303149086000BF30480C
:10041000006800F4003000900198401C01900098A2
:1004200018B90198B0F5A06FF1D12948006800F41F
:10043000003010B10120009001E0002000900098F1
:10044000012843D12348006840F01000214908608A
:100450000846006820F0070008600846006840F081
:10046000020008601A484068194948600846406818
:1004700048600846406840F480604860084640682C
:1004800020F47C1048600846406840F4E81048605A
:100490000846006840F08070086000BF0C480068A3
:1004A00000F000700028F9D00948406820F00300EF
:1004B000074948600846406840F00200486000BFB5
:1004C0000348406800F00C000828F9D10CBD00007A
:1004D000001002400020024010B500F001F810BDED
:1004E00010B50D48006840B10B480068401E0A492D
:1004F000086010B9012009490870002408E004EBE5
:100500004401074A02EB810000F026FD601CC4B2E2
:10051000042CF4DB10BD0000080000200C000020BB
:100520008C00002010B51348006840F0010011490C
:10053000086008464068104908400E49486008466F
:1005400000680E4908400B4908600846006820F41E
:10055000802008600846406820F4FE0048604FF4A0
:100560001F008860FFF744FF4FF0006004490860F7
:1005700010BD0000001002400000FFF8FFFFF6FE73
:1005800008ED00E07047000010B50121264800F09A
:1005900064F818B10121244800F050F802212248E3
:1005A00000F05BF858B102211F4800F047F8002224
:1005B00002211D4800F062F81C48006880470421B1
:1005C000194800F04AF858B10421174800F036F8ED
:1005D00000220421144800F051F8154800688047B3
:1005E0000821114800F039F858B108210E4800F0F0
:1005F00025F8002208210C4800F040F80D4800685A
:1006000080471021084800F028F858B1102106480A
:1006100000F014F800221021034800F02FF80648DB
:100620000068804710BD0000000400401400002056
:10063000180000201C00002020000020CA43028275
:10064000704721B1028842F00102028004E0028872
:100650004FF6FE731A400280704730B50246002004
:1006600000230024158A05EA0103958905EA01049F
:1006700013B10CB1012000E0002030BD1AB1838914
:100680000B43838102E083898B4383817047018917
:100690004FF6F872114001817047000070B50024D8
:1006A00000220023058C4FF6FF6635400584028C3E
:1006B0008388848B4FF68F752C404FF6FC752C4049
:1006C0000D882C434FF6FF552A400D894FF6FF76D3
:1006D00006EA05252A434D8806EA05252A43154DD5
:1006E000A84202D0144DA8421DD14FF2FF752A40F6
:1006F0004D894FF6FF7606EA05252A434FF6FF356A
:100700002A408D8806EA05252A434EF6FF752B40C0
:100710004DF6FF752B408D8906EA05152B43CD89D3
:1007200006EA05152B4383808483CD888587028460
:1007300070BD0000002C0140003401400021018008
:1007400041808180C180018141818181C181704767
:10075000002202881D4B98420ED01D4B98420BD0B0
:10076000B0F1804F08D01B4B984205D01A4B9842ED
:1007700002D01A4B984204D14FF68F731A404B881F
:100780001A43174B984207D0164B984204D04FF6A5
:10079000FF431A40CB881A4302808B8883850B88DD
:1007A00003850A4B98420BD0094B984208D00E4B58
:1007B000984205D00D4B984202D00D4B984201D182
:1007C0000B7A03860123838270470000002C0140CE
:1007D000003401400004004000080040000C0040CC
:1007E000001000400014004000400140004401405F
:1007F0000048014010B540F226610C4800F08FF827
:1008000020B140F22661094800F012F840F225516B
:10081000064800F084F840B140F22551034800F04A
:1008200007F8024800F012F9C4B210BD00380140C8
:1008300010B50022002340F66A14A14200D100BF87
:100840000A1201249440A3B2DC43048010BD21B1FC
:10085000828942F40052828104E082894DF6FF735E
:100860001A4082817047000010B504462048844237
:1008700009D101218803FFF741FD00214FF4804099
:10088000FFF73CFD32E01B48844209D101214804B6
:10089000FFF714FD00214FF40030FFF70FFD25E0B6
:1008A0001548844209D101218804FFF707FD002182
:1008B0004FF48020FFF702FD18E01048844209D170
:1008C0000121C804FFF7FAFC00214FF40020FFF7D4
:1008D000F5FC0BE00A48844208D101210805FFF726
:1008E000EDFC00214FF48010FFF7E8FC10BD000084
:1008F000003801400044004000480040004C0040E7
:100900000050004002460020B1F5007F00D100BF3A
:1009100013880B400BB1012000E00020704770B538
:100920000246002400230025002040F66A16B1424A
:1009300000D100BFC1F3421501F01F03012606FAE2
:1009400003F3012D02D19689334006E0022D02D136
:10095000168A334001E0968A33400C12012606FACB
:1009600004F41688344013B10CB1012000E00020DB
:1009700070BD00002DE9F04786B005460E46002404
:10098000A24600BFA1460027B08900B100BF2F4694
:100990002C8A4CF6FF700440F08804432C82AC890A
:1009A0004EF6F3100440B08831890843718908433A
:1009B0000443AC81AC8A4FF6FF400440B089044345
:1009C000AC8201A8FFF7AAFC1F48874202D1DDF8DC
:1009D00010A001E0DDF80CA0A88900F4004040B1AF
:1009E0000AEBCA0000EB0A1031684900B0FBF1F8CD
:1009F00007E00AEBCA0000EB0A1031688900B0FB7F
:100A0000F1F86420B8FBF0F004012009642101FB37
:100A10001089A88900F4004040B1322000EBC900E1
:100A2000B0FBF1F000F00700044308E0322000EBD7
:100A300009106421B0FBF1F000F00F0004432C8199
:100A400006B0BDE8F0870000003801400146888804
:100A5000C0F308007047C1F30802828070470000AD
:100A60000FB4054B10B503A9044A029800F01AF818
:100A700010BC5DF814FB00000912000824000020DF
:100A800002E008C8121F08C1002AFAD17047704757
:100A9000002001E001C1121F002AFBD1704780F342
:100AA000108870472DE9F84F9946924688460546CA
:100AB000002706E025280AD051464A4690476D1C7B
:100AC0007F1C28780028F5D13846BDE8F88F002330
:100AD00015F8011F18462E2915D115F8011F0423FA
:100AE0002A290DD06FF02F022978A1F13004092CAA
:100AF00009D800EB800002EB400008446D1CF3E7CE
:100B000058F8040B6D1C2A78002ADDD0632A07D020
:100B1000732A0FD0104651464A4690477F1C2AE060
:100B200018F8042B8DF8002000218DF801106E4676
:100B3000012103E058F8046B4FF0FF315A074FF0E2
:100B4000000401D409E0641C84420BDA8C42FADB15
:100B5000325D002AF7D105E0641C8C42FCDB305D7D
:100B60000028F9D1274404E016F8010B51464A4603
:100B70009047641EF8D26D1CA3E710B500F0FAF898
:100B800010BD000010B52248007820B1012808D01F
:100B900002283AD11EE001201E4908701C49087045
:100BA00034E01C480078002805DD00201949087051
:100BB000FA2000F0C2FB00F0BBFB002806DD02209B
:100BC0001349087001201349087002E0124988682F
:100BD00080471BE00F480078002805DD00200D4904
:100BE0000870FA2000F0A9FB00F0A2FB002808DD45
:100BF0000120074908700749087008A0FFF730FF77
:100C000002E00549C868804700E000BF00BF10BD92
:100C10000100002005000020500000204661756C96
:100C20007421200A0000000010B52348007820B18C
:100C3000012808D002283CD11FE001201F4908707C
:100C40001D49087036E01D480078002806DD0020A8
:100C50001A4908704FF4FA7000F06FFB00F068FB5F
:100C6000002806DD0220144908700120134908708D
:100C700002E01349886880471CE01048007800288B
:100C800006DD00200D4908704FF4FA7000F055FBA6
:100C900000F04EFB002808DD0120074908700749D5
:100CA000087008A0FFF7DCFE02E00549C86880472D
:100CB00000E000BF00BF10BD0100002003000020C5
:100CC0005000002049646C6521200A0010B52348BB
:100CD000007820B1012808D002283CD11FE0012073
:100CE0001F4908701D49087036E01D48007800282B
:100CF00006DD00201A4908704FF47A7000F01DFBE1
:100D000000F016FB002806DD0220144908700120BF
:100D10001349087002E01349886880471CE01048B6
:100D20000078002806DD00200D4908704FF47A7025
:100D300000F003FB00F0FCFA002808DD0120074961
:100D400008700749087008A0FFF78AFE02E005490D
:100D5000C868804700E000BF00BF10BD0100002050
:100D6000040000205000002052756E6E696E6721ED
:100D7000200A000000B585B00021684600F078FA2E
:100D8000142269460248FFF7CFF905B000BD000004
:100D90005000002010B50A48007820B1012805D085
:100DA000022809D105E0FFF73FFF06E0FFF78EFFBD
:100DB00003E0FFF7E7FE00E000BF00BF10BD00004A
:100DC0000000002010B500F003F8FFF7E3FF10BDAE
:100DD000084800780849087008480078097888426F
:100DE00006D00548007805490870002004490870BD
:100DF00070470000020000200000002006000020D4
:100E0000010000200146042901DB0020704701EBAE
:100E10004100084A02EB80004078012808D10020F8
:100E200001EB4102034B03EB820250700120EDE71E
:100E30000020EBE78C00002008B501210420FFF71B
:100E40004DFA10208DF80300ADF8000003208DF856
:100E5000020069461548FFF78BF910208DF8030052
:100E60002020ADF8000003208DF8020069460F48ED
:100E7000FFF77EF910208DF803004020ADF8000048
:100E800003208DF8020069460848FFF771F9102029
:100E90008DF803008020ADF8000003208DF80200DB
:100EA00069460248FFF764F908BD000000080140E8
:100EB00010B5FFF7C1FF00F001F810BD00B589B013
:100EC00001210846FFF7EAF908A92248FFF750F97F
:100ED00001210420FFF702FA0420ADF820001820B9
:100EE0008DF8230003208DF8220008A91948FFF788
:100EF0003FF94FF08040FFF7CAFB6320ADF81800C0
:100F00002320ADF814000020ADF81A00ADF816004B
:100F10008DF81C0005A94FF08040FFF719FC01A8CF
:100F2000FFF70CFC6020ADF804000020ADF80C00C9
:100F30000120ADF806000020ADF80A0001A94FF02D
:100F40008040FFF7ABFB01218807FFF77AFB09B070
:100F500000BD000000080140416851B14168491ED0
:100F6000416031B9012141700178012901D18168C5
:100F70004160704770B504460D46042C06DB114AEB
:100F800011A118A0FFF76CFD00BFFEE70120FFF7DD
:100F900086FD04EB44001B4901EB8000456004EB37
:100FA000440001EB80008560002004EB4401154AF9
:100FB00002EB8101487004EB440102F82100FFF7C5
:100FC0006EFD70BD481300082E2E5C436F64655C97
:100FD0006273705C7372635C6273705F74696D6579
:100FE000722E63004572726F723A2066696C6520DA
:100FF00025732C2066756E6374696F6E20257328C7
:10100000290D0A008C0000200146002011B9044A75
:10101000D26804E0012902D1024A12680020704718
:10102000001001400C0C014010B500F05DF800F01C
:10103000A9F8FFF73DFF10BD08B501211020FFF70B
:101040004DF9002000F02CF84FF40050ADF80000EE
:1010500010208DF8030003208DF802006946024835
:10106000FFF786F808BD00000010014008B5012117
:101070000820FFF733F9012000F012F84FF4007058
:10108000ADF8000010208DF8030003208DF8020059
:1010900069460248FFF76CF808BD0000000C0140EB
:1010A00020B94FF40051044A516104E0012802D1F3
:1010B0004102024A1160704700100140140C0140C7
:1010C00028B90749096941F40051054A116101280D
:1010D00005D10449096841F40071024A1160704762
:1010E00000100140100C014070B5002016E00021F6
:1010F00000EB40021F4B03EB8202516000EB400209
:1011000003EB8202916000EB400203EB820251701C
:1011100000EB400203F82210411CC8B20428E6DBB1
:10112000154909684FF47A73B1FBF3F2B2F1807F8D
:1011300000D31DE022F07F41491E4FF0E0235961AA
:1011400059170F23002907DA1C07260E0B4C01F054
:101150000F052D1F665503E01C07250E084C65542E
:1011600000BF00214FF0E02399610721196100BF02
:1011700070BD00008C0000202800002018ED00E069
:1011800000E400E000B585B001210420FFF7A6F8D7
:1011900001214804FFF782F81948FFF765FB042096
:1011A000ADF8100003208DF8120018208DF8130000
:1011B00004A91448FEF7DCFF0820ADF81000042055
:1011C0008DF8130004A90F48FEF7D2FF4FF4E13069
:1011D00000900020ADF80400ADF80600ADF808005E
:1011E000ADF80C000C20ADF80A0069460448FFF782
:1011F000C1FB01210248FFF72AFB05B000BD00003A
:10120000004400400008014070B504460D4600BF90
:1012100040210548FFF776FB0028F9D0E1B20248EB
:10122000FFF719FC204670BD004400404FF4A06059
:10123000FFF72AF8FFF7F8FE00F006F8FFF79DFC2D
:1012400001E0FFF7BFFDFCE710B500F039F810BD75
:1012500010B500240020FFF7D7FE0446204610BD3D
:1012600010B500240120FFF7CFFE0446204610BD34
:1012700070B505460C46022C01DB00BFFEE704EB0F
:101280008400044A02EB800114222846FEF74CFF3A
:1012900070BD00006400002010B50020FFF700FFC3
:1012A00010BD10B50020FFF70BFF10BD10B50120D9
:1012B000FFF7F6FE10BD10B50120FFF701FF10BDCE
:1012C00010B5002011490870114848601148886025
:1012D0001148C860114808610120087510490B4881
:1012E00081611049C16110490162104941620024C5
:1012F00008E004EB8401054A02EB8101486880475D
:10130000601CC4B2022CF4DB10BD0000640000209D
:1013100039100008A31200089912000851120008A1
:101320006D100008B7120008AD1200086112000825
:1013300010B50020FFF766FD10BD10B5044621462C
:101340000020FFF717FE10BD6273705F5374617267
:101350007454696D6572006273705F537461727466
:101360004175746F54696D6572006273705F537478
:101370006F7054696D6572009813000800000020BA
:1013800050000000800A0008E81300085000002008
:1013900070040000900A0008000000000000000037
:1013A000000000000000000000000000000000003D
:1013B000000000000000000000000000000000002D
:1013C00000A24A0400000000000000000102030423
:1013D00006070809000000000102030401020304DB
:0813E0000607080902040608D3
:04000005080000ED02
:00000001FF
